:020000040000FA
:060000000219FD0200C818
:03000B0002008D63
:03002B000200923E
:03005B000202C6D8
:030073000200B5D3
:100080000406080C10182030406080A0C0C28D0506
:100090004032C0D0C0E0C2CF0541E5646009E563ED
:1000A000600575630001B0756301E52360021523E7
:1000B000D0E0D0D032C2AF53E67F7592FA7593FF8D
:1000C000C22053917FD2AF32C0D0C0E0C0F0D2D3B3
:1000D0005388EFA88AA98CAA40308D010A758A003E
:1000E000758C00754000438810E564700AC3E833DE
:1000F000F8E933F9EA33FA30331FE8C4540FFAE968
:10010000C454F04AFAC3132AFAC3E833F8E933F9BE
:10011000E82AFAE93406FB216C30320FC3E833E9F0
:1001200033FAE82AFAE93400FB216C303115E8751E
:10013000F056A4AAF0E975F056A42AFAC5F03400E6
:10014000FB216CC3EA13FAE913F9E813F8E875F038
:1001500056A4AAF0E975F056A42AFAC5F03400C3F3
:1001600013FBEA13FAC3EB13FBEA13FAC3EB941283
:100170005006C3EB9406501A0522E52270021522A0
:10018000C3E522940A500241BC7552007A007B00FC
:10019000418DE522600215223035067C007D082164
:1001A000ACAC31AD32303A04AC33AD34C3EA9CFA76
:1001B000EB9DFB9208AE5EAF5F303A4250072034B1
:1001C00009D23421CA303402C234303404AE60AFB4
:1001D00061203902B234C3EA33FAEB33FBA2085090
:1001E0000AEAF42401FAEBF43400FBC3EA9450FA6F
:1001F000EB9400FB501478007A007B00410AA208BF
:10020000500878007A007B004169E5255403601BA3
:10021000202A18E55B33F9EB7007C3E99A4002E93D
:10022000FAE53CC4332AFAEB3400FBEA8EF0A4F979
:10023000AAF0EB8EF0A42AFAC5F03400FBC3EB134E
:10024000FDEA13F8C3ED13FDE813F80FEF14600493
:10025000C3E833F8C3E933EA33FAEB33FBDFEDEB02
:1002600030E30678FF7AFF7B078852D230C3E894E8
:10027000404002D221C3E559FC955A4003AC5AC311
:10028000EC95525008EC75F008A4FAABF0EAF4F8DB
:10029000EBF45407F9C3E89428FAE99400FB5004FE
:1002A0007A007B00885489558A568B5775230AD06B
:1002B000F0D0E0D0D053F7DF43F7403275230AD0B7
:1002C000F0D0E0D0D032C0D0C0E0D2D3A8F9E55809
:1002D00030E107E5FA30E2076114E5FA30E235C3B0
:1002E000E55513F8E55413F5FB88FCC3E55713F8FF
:1002F000E55613F5E988EA85555853F7BFC3E5522B
:10030000940140057553006114E5532401F55350E1
:10031000037553FF53F7DFD0E0D0D032790180145A
:1003200079038010790A800C791E80087964800432
:1003300079C880007817E4D5E0FDD8FAD9F6227A9A
:10034000147B7880127A107B8C800C7A0D7BB480C1
:10035000067A0B7BC880007902E4C293D5E0FDD217
:1003600092D5E0FDC292D5E0FDD293D5E0FDE92023
:10037000E002D29030E002D294E562D5E0FDE920BF
:10038000E002C29030E002C2947496D5E0FDD9C973
:10039000EAF8D5E0FDD8FBDBBEC2932278FFC2218C
:1003A00020283D202912D221C3E548940A4009C3E0
:1003B000E55294405002C22179A1E76023E54860EC
:1003C0001F74FF8548F084853FF030290375F005E0
:1003D000A4F8C5F0600278FFC3E8955B5002A85B03
:1003E000885A22C3E54794A0E5489400E55A500393
:1003F0001461F4046002F55A2275E89022055CC38A
:10040000E55C94084055E5E820ECF2A8BDA9BE756E
:100410005C00E9FA79A0E76041EA7006E55D6018E2
:10042000800CC3E8955D600EE55D5005600A1480A0
:10043000070460FA8002E55DF55DC394F6401B7524
:1004400059C0C394064013755980C39406400B7578
:100450005940C39406400375590022E559241050B1
:100460000274FFF55922743279A687F0A4C5F0A270
:10047000F733F8C3E895594002A859885B227547BD
:10048000007548F022C2AF75C800A8CCA9CDAA411A
:1004900030CF010A75C804D2AFC3EA13FAE913F9E1
:1004A000E813F8AB42AC4388428943C3E89BF8E9C0
:1004B0009C20280A547FF9302C02A19F81FCAD4476
:1004C0008A44F9EA9D547FFA600478FF79FFAE45CB
:1004D000AF468B458C46A842A943C3E89EF8E99FE6
:1004E000F9C3E54813FBE54713FAE82AF547E93B6A
:1004F000F54850067547FF7548FFA146AA47AB4827
:10050000AC47AD487E047F02C3EB9404400A1E1F33
:10051000C3EB940840021E1FC3ED13FDEC13FCDE79
:10052000F7C3EA9CFAEB9DFBEF6009C3E913F9E816
:1005300013F8DFF7EA28FAEB39FB8A478B485006B5
:100540007BFF8B478B48C3EB94025002D22C3028A0
:10055000047F03A1717892E6FFC3E53D94824011C8
:100560000FC3E53D94A040010FC3EF940640027F06
:10057000057E02E548C4540FF9E548C454F0F8E597
:1005800047C4540F28F8C3E89EFAE99400FB4009D9
:10059000C3EA9401EB940050047A01E4FBA1EBAAB6
:1005A00047AB48EBC4FEEAC4540F4EFCC3EA9CFAC6
:1005B000EB9400FBC3E813C313F8EA28FAEB34000A
:1005C000FB8A478B48C3EB94024002C22C7802EBB3
:1005D000C4FE7B00EAC4540F4EFAC3EA98FA400501
:1005E000C3940150027A017892E6FF30200280FB2A
:1005F000854E92854F93D22043E680C3E49AF8E477
:100600009BF9C3E833F8E933F9302C02C17DE8FAED
:10061000E9FBD3E913FDE813FC884E894FC3EF943F
:10062000036037EF20E00CE82CF8E93DF9ECFAED37
:10063000FB8013E828F8E939F9C3E82401F8E93424
:1006400000F97AFF7BFFC3EF9403400E8A508B5171
:10065000884A894B8C4C8D4DC1B1885089518A4A4A
:100660008B4B8C4C8D4D3028127550F07551FF75A9
:100670004CF0754DFF754EF0754FFFC1B1E8FAD3E0
:10068000E813FC884EC3EF94036020EF20E007E8F6
:100690002CF8ECFAC19DE8282401F87AFFC3EF9406
:1006A0000340088A50884A8C4CC1B188508A4A8CD1
:1006B0004C302002C1B1753A02D22043E680E525D4
:1006C0005403602DA847A948C3E913F9E813F8308B
:1006D0002804E92440F9C2AF53E67F759100C3E4D2
:1006E00098F594E499F595759104D22043E680D26B
:1006F000AF22D222754900752000302B03752040AF
:10070000800ED222754900752040302B03752000E1
:1007100078017901202C20E52554036002C222795A
:1007200014E548C313700104F8C39414400278140C
:10073000302804781B791BC3E833F8C3E933F92068
:100740002010E549600C302803D53A04D224E1C7D3
:10075000D1B90549E59B5440B52002E1B1302809E3
:1007600008C3E899400118E13F20220A08C3E8992C
:100770004002E110E13FC222C2AF53E67F75910013
:10078000302C127594007595FC759104D22043E6C7
:1007900080D2AFE110AE47AF48C3EE33FEEF33FF78
:1007A00050047EFF7FFFC3E49EF594E49FF595E13E
:1007B00089C3E53994015002E110302202E110D8DA
:1007C00002E1C5E13FC224C2AF53E67F75910085C7
:1007D0005094855195759104854A92854B93D2200A
:1007E00043E680D2AFE5255403600720290205398E
:1007F000801030240D202B0A20220715811581023C
:100800000EF22278003021053022027801E53D7594
:10081000F007A4F9E5F028F5F0E9A2F013A2F1132E
:10082000A2F213F53DC394785003753D78C3E53DBE
:10083000953E400BD223C290C292C29475D53F30F0
:10084000200280FB854C92854D93D22043E6802286
:10085000203810C2AFC293D29175D50FD2AF759F19
:10086000032124C2AFC293D29575D53CD2AF759FF8
:10087000032124203811C2AFC29475D533D291D24E
:10088000AF759F13020924C2AFC29075D533D295BC
:10089000D2AF759F23020924203810C2AFC291D273
:1008A0009575D533D2AF759F238079C2AFC295D2EB
:1008B0009175D533D2AF759F138069203811C2AFBF
:1008C000C29275D53CD295D2AF759F03020924C25E
:1008D000AFC29275D50FD291D2AF759F0302092492
:1008E000203810C2AFC295D29375D53CD2AF759F58
:1008F000138031C2AFC291D29375D50FD2AF759F1D
:10090000238021203810C2AFC29075D50FD293D268
:10091000AF759F23800EC2AFC29475D53CD293D2DF
:10092000AF759F13C22322C290C292C294C291C2D9
:1009300093C29575D53F22788076FF0876FF0876BA
:10094000FF0876FF0876FF0876FF0876090876FF2D
:10095000087601788C76010876FF0876FF0876FF26
:100960000876FF0876FF0876030876FF0876FF080A
:1009700076FF0876250876D008762808765008761F
:10098000040876FF0876020876FF08767A0876FF74
:100990000876010876010876FF0876FF08760008D9
:1009A000760022FA75F00CA4ABF0EAC333F87401B8
:1009B00033F9E8C333F8E933F9E8C32BF8E9340035
:1009C000F9E8C333F8E933F9227888E6C39403D20F
:1009D0003A5002C23AC238E630E102D238A2389226
:1009E000397886E6149000809378A6F67886E6F546
:1009F0003FC394025003753F02789CE6753EFFB4F6
:100A00000203753EA0B40303753E827896E631A3D7
:100A100088318932789EE631A3883389347897E625
:100A200031A3883589363127223035117A007B0091
:100A30007CFF7D007E0051908B5F8A5E22303A22DF
:100A40007896E6FA7B00789EE6FC7D00C3EA33FAEE
:100A5000EB33FBC3EC33FCED33FD7E0A51908B612D
:100A60008A607896303A02789EE6FA7B007897E6BC
:100A7000FC7D007E00303A10C3EA33FAEB33FBC34F
:100A8000EC33FCED33FD7E0A51908B5F8A5E2222AF
:100A9000C3EC9EFCED9400FDC3EC9AFCED9BFDC302
:100AA000EC9423ED940050047C237D00C3EC94FF70
:100AB000ED940140047CFF7D017BFF0B7A000AEA84
:100AC0007009C3EC33FCED33FD41BBEC8AF0A4AEFE
:100AD000F0ED8AF0A42E947C40E4EAF460DD22D2AA
:100AE0003551291203287A007B007C10120320E57F
:100AF000522AFA74003BFBDCF37C04C3EB13FBEAE1
:100B000013FADCF7FFEB60027FFFC2355129227830
:100B1000A5E6F954037000E9540C7000E9543070F4
:100B200000E954C0700022E5EF20E60375200005BF
:100B300020903FFFE520146006901DFF1460009395
:100B400004600375EF127597DE7597AD7581C0432C
:100B5000FF8012031C75EF0275A90031277580FF15
:100B600075F1F075A4007580FF75D4FF7590007560
:100B7000F23F75A53F75900075D53F75A60175E3E9
:100B80004075E2023127E4F8F6D8FD3137F13378C9
:100B9000988662753001C2AF12033012033F120310
:100BA0002812034512032812034B120328710FC2A7
:100BB000AF78FA79FA308507D9FBD8F7021C0031F3
:100BC000C9512978988662312775A91375A71075C0
:100BD000C10075A70075640075E405758811758EF0
:100BE0000475890975C80475910475D84075D908CC
:100BF00075F782759E0375960275DA4275DB42754C
:100C0000A82375E69075F310759B80759D0075D1CE
:100C10002C75BCC075BB1075E88075B20112031C41
:100C2000D2AF753C00C230120330C23175220012BF
:100C3000032CC3E522940A4024D231C2327522002B
:100C400012032CC3E522940A4013D232C233752218
:100C50000012032CC3E522940A4002D2331203206F
:100C6000203003020BAFC2AF12033F12033F120347
:100C70003FD2AF120330303A02A109120320788C20
:100C8000E6C394015002A109E530C394015002A1CA
:100C9000097F02D235512912032CC2AFC235512926
:100CA000AE52C3E552947FD2AF405E12031CC2AF76
:100CB000120351D2AFDFDC51DFC3EF7897F6120396
:100CC00030F16D1210107F0AD235512912032CC257
:100CD000AFC2355129AE52C3E552947FD2AF50E630
:100CE00012031CC2AF12033F12032412033FD2AF00
:100CF000DFD651DFEF24037896F6120330F16D1240
:100D0000103F12032C512961AF12032C7801303AA5
:100D1000027805C3E5529840028176C2AF120351B2
:100D2000120351120351D2AF120330753000E4F5B3
:100D300037F5380537E537F4703E0538789AE678A8
:100D400019146012783214600D787D14600878FAF6
:100D5000146003753800C3E53898401C312712032E
:100D60001C153875370078998662C2AF120351D2CC
:100D7000AF7898866212032C120324E52370026177
:100D8000AF7801C3E5529840AA12032CE523700303
:100D9000020BAFC2AF3127E4D2AFE4F55CF524F526
:100DA00025F53D755C0812031C1203F9E5E820ECFB
:100DB000FBA8BDA9BEE97001F8885D1203FD755C52
:100DC00008C2AF7559FF120466855B59855B5AD21C
:100DD000AF75A71075C13075A70075A903756401BB
:100DE000303A07C238303402D238D228753900116F
:100DF000E0310312047E12048512047E120485126F
:100E0000047E120702110311501204851206F2200B
:100E10002C0312039C302C031203E31103117312F1
:100E20000485120702110311981204851206F211AB
:100E30000311BB120485120702110311E01204858D
:100E40001203F91206F2110331031203FD12048595
:100E5000302827855B5979187A0CC3E53999400EFB
:100E6000C228D2298A3B855B59855B5A800CC3E531
:100E70005294014003020E02C1FA30291C202B19A2
:100E8000E53B147006C229D22AC102F53BC3E552E4
:100E900094014003020E028061753C0078FA79A447
:100EA000E760027803C3E55398504FE523604B3069
:100EB0003A17203805203407800F303402800A208A
:100EC0002B07D22B855B59C12C78F0302B05855B25
:100ED000597820C3E548985003020E02302B1BC2FC
:100EE0002BC238303402D238D229753B12855B5977
:100EF000C102053CE5526002C1FD753C00C2AF3144
:100F00002775240075250075A91375A71075C100F4
:100F100075A700756400D2AF12032C312778A4E6C0
:100F20006006D291D293D295C3E53C94044002610D
:100F3000AFA12E901A0D7820F1A6E520B4550AA392
:100F4000F1A6E520B4AA0280063137F16D801D902C
:100F50001A0378807B0AF1A6A308DBFA901A0F78AF
:100F60008C7B1AF1A6A308DBFA901A2922C2AFF1F2
:100F7000E5F1BF901A007410F1ABA37401F1ABA3BB
:100F80007420F1AB901A0378807B0AF1AAA308DBE6
:100F9000FA901A0F788C7B1AF1AAA308DBFAF1F801
:100FA000F1D6901A2922E493F622E6438F01538F5B
:100FB000FD75EF0275B7A575B7F1F0538FFE2243AB
:100FC0008F02438F0175EF0275B7A575B7F1901ABF
:100FD0000DF0538FFC22901A0D7455F1AB901A0E40
:100FE00074AAF1AB227A3079D07820901A40F1A619
:100FF000E520F709A3DAF7227A3079D0901A40E792
:10100000120FAB09A3DAF8227C05120330DCFB22B5
:10101000C2AF12033F12034512034B1203511203D6
:101020002412033F12034512034B120351120324EF
:1010300012033F12034512034B120351D2AF22C2D7
:10104000AF12035112034B12034512033F12032444
:1010500012035112034B12034512033F12032412D1
:0E106000035112034B12034512033FD2AF227D
:1019FD00020B27100120FFFFFFFFFFFF09FF01FF73
:101A0D0055AA01FFFFFFFFFF03FFFFFF25D0285061
:0D1A1D0004FF02FF7AFF0101FFFF0000FF40
:101A400023475F485F3230232020202020202020A1
:101A500023424C48454C492445464D3842323123B7
:101A60002020202020202020202020202020202076
:101C0000C2AFC2D37597DE7597AD7581C075A90057
:101C100043FF80752438752503B1C875EF0243F181
:101C20002053A4DFD28575D4FF75E3407DFA780395
:101C300079E67C10752200752300901DD57B067512
:101C400024987525013085028145208508D8FBD967
:101C5000F9DCF781B7308508D8FBD9F9DCF781B713
:101C6000B188E493A3C39A6004DDC381B7DBDBB121
:101C70007A6002812E7B08E493FAA3B15BDBF87AE9
:101C800030B15B752200752300B17AEAFCEBFDC32D
:101C9000ED94FE400EB17A8A278B28ED30E0048A5D
:101CA000828B83B17A7AC270D8C3ED94FE601350F0
:101CB000CEBD0023EC60097520007521FF020000F5
:101CC0008100A827A9280809D804D90281D4B17EA7
:101CD000EAF281C80D81A3C3ED94035047EDA2E061
:101CE00092007AC5C3E5829400E583941C5092204B
:101CF0000010438F02438F0175B7A575B7F1F0301F
:101D0000001DA827A9280809438F01538FFDD80477
:101D1000D902A11FE275B7A575B7F1F0A3A10E53C3
:101D20008FFC817F7AC1BD030CE493A3FAB13FDC41
:101D3000F8B137817F8181AA22AB23B15BEBFAEA4C
:101D40006222752608C3E52313F523E52213F52245
:101D500050066323A0632201D526EAB1C8B1C87535
:101D6000260AEAF4200102D285300102C285B1C8F8
:101D7000C3134002C201D526EB22B17EEAFB2085C7
:101D800002A17E308502A183752608AE24AF25C34B
:101D9000EF13FFEE13FEB1CCB1C8C3EA13308502D6
:101DA0004480FA30E703632201C3E52313F523E5FA
:101DB0002213F52250066323A0632201D526D9E51C
:101DC0002265236523F52222AE24AF250E0FDEFE09
:101DD000DFFCD20122424C48656C6934373163E83C
:031DE000B2060147
:00000001FF
